:10014000021D800A0A5052494E540D0A80140A506A
:1001500052494E540D0A801E205052494E542022BE
:10016000544154544C4554414C45204D4F44454C0A
:100170002023223B0D208028105052494E54204D00
:100180004F44454C0D1080320A5052494E540D0ACE
:10019000803C225052494E5420222020532F4E2082
:1001A000222C20534E25313030303030303030303A
:1001B0000D2280462A5052494E542022284329209D
:1001C00031393838204F4E53455420434F4D505508
:1001D00054455220434F52502E220D2A80500A502F
:1001E00052494E540D0A805A2F5052494E542022E3
:1001F0005454424153494320222C564552532F31E7
:1002000030302C222E222C2330322C5645525325AE
:0D0210003130300D2F8064084E45570D0829
:10C000008E00FFBDF5CA8621BDF8DEBDC0C842C0A6
:10C010002743C03044C03946C07B4DC12B50C29F1E
:10C0200052C27653C0AA00BDF8DE717F147EF93487
:10C03000BDF8DEBDF5CA7EC6FEBDC0E33CBDFA62FA
:10C04000BDF903383CC610A600BDFA67BDF9070864
:10C050005A26F4BDF90338C610A60081202C0286AA
:10C060002E817F2F02862EBDF8DE085A26EBBDF505
:10C07000CABDC128812E26C47EC000BDF8DEBDF930
:10C0800007BDC0F6183C862CBDF8DEBDC0F6DD56F7
:10C09000862CBDF8DEBDC0F637BDF5CA3238A70024
:10C0A000089C5626F9A7007EC000BDC0E3BDFA6219
:10C0B000BDF903A6009753BDFA67BDF903BDC0F6ED
:10C0C000E700BDF5CA0820E5383CBDC128A100271E
:10C0D000096D0027F308080820F3333336EC011804
:10C0E000326E00BDF8DEBDF9077F00527F0053BD00
:10C0F000C0F6187EF5CABDC128812E26037EC00079
:10C10000810D2603DC5239803025EB810A25088019
:10C110000725E3811024DF9746BDFA6FDC52050541
:10C120000505DB46DD5220CE7EF8A1BDF8DEBDF56B
:10C13000CABDF86C26FB71F8175FF740005CC108B8
:10C1400027057C001720F371F8175FF140002738AE
:10C15000B64000363771F817CEC1754FBDF44B327B
:10C160008A30BDF8DECEC17D4FBDF44B328A30BD82
:10C17000F8DE7EC0003A2042414E4B20002052455E
:10C1800041445320415320005CC10827057C00171F
:10C1900020B971F817CE4002EF001805847F8B405C
:10C1A000188C400026F2CE4002AC002743DF46EE5A
:10C1B00000DF4871F817BDF5CACEC1E14FBDF44BA1
:10C1C0009648BDFA679649BDFA67CEC1E64FBDF401
:10C1D0004B9646BDFA679647BDFA6771F8177EC061
:10C1E0000053454520002041542041444452200042
:10C1F0001805847F8B40188C400026AD8601974639
:10C2000071F81796179A469717CE40004F5FED00CA
:10C21000EC00261E4353ED00A300261F08088CC027
:10C220000026EB7C00469646810826D771F8177EDB
:10C23000C000CC0000ED00EC002007CCFFFFED00BB
:10C24000EC003C373671F817BDF5CACEC26B4FBD56
:10C25000F44B323318BDFA628640BDF8DE383CBD7F
:10C26000FA6238EC004353ED0020F842495420456F
:10C2700052524F522000BDF8DEBDF5CA4F3632365D
:10C28000BDF64ADE56BDFA62BDF903324C36814036
:10C290002709840726E8BDF5CA20E3327EC000BD29
:10C2A000F8DEBDF5CA7F0053BDC0F6C43F37BDF907
:0DC2B00003BDC0F6DD5632BDF69A7EC0001B
:10C4000000000030303030303030303030300D54BB
:10C410004154544C4554414C45204D4F44454C20CB
:10C420003220202843292031393838204F4E5345B7
:10C430005420434F4D505554455220434F52502E97
:10C440000D4C495354CB15545952554ECAB3505202
:10C45000452A52554ECAAC462452454D494E44CF0A
:10C4600091465245D73B414F4E454F4ED7DE414155
:10C4700041454F4646D7D942424E455854C931549A
:10C480004F4C4554CE785641524946CDBC4E4F5440
:10C4900045474F544FCAFD454E474F535542CD6710
:10C4A0005352455455524ECD90464F52C8A9474518
:10C4B000544255525354CE885853544F5245CECBC4
:10C4C0004150534554D392564150434C52D3FC549F
:10C4D0004553444FDAB231313143414C4CDBDD320C
:10C4E00032434F554E54DD0F45534C454550D31400
:10C4F000525550524F47DB755855474554D4E9447F
:10C5000046544F4E45D75652535553454E44D4602A
:10C510002F4F4E455252D63F2341534DDE7F4A4E58
:10C520004B52454DCDAD41524B5052494E54CC46E5
:10C5300053584D4954D806574F53544F50CAA654D8
:10C540004F4954455854D65F4F4F54455854D6F32D
:10C55000475354494D45D823405254494D45D97904
:10C56000405653544F5245DC6056474554DC9A338D
:10C5700033494E505554CDE138585348414B45D777
:10C58000E94F46464C44D156454F4E4C4F4144DD51
:10C590004D44494DDCCC5245414E4557CA924F4C13
:10C5A00044434F4EDCEE444545CE72544FC8CC4612
:10C5B000524F4DF2AD53544550C8E14154C8E74382
:10C5C00048414EE5415459474554E57D26474F5073
:10C5D000494EE5FB544845534449E96D202020501D
:10C5E0004552494F44EA54414253E52C4245455394
:10C5F0005152E67C47415454454D50E73148495328
:10C60000494EE7F24F46464153494EE85E4E554388
:10C610004F554E54E9C0454C4F47EB11494E4745E5
:10C620005850ECCC495245424154E716544F5056AD
:10C63000455253E9525A59534EE95E50495A454DB5
:10C640004F44454CE94953E4F83DE37E252F2F2A1A
:10C65000343E3DE34F2F233C2F3E3CE35A7E2F2AAE
:10C660003C3C3EE35A2B3D2D3E3EE36C454E442E72
:10C670002E3C3DE3753F2F3E3E3CE3853C3E3C3E39
:10C680003CE38C8EBFFF7F00760E86FF9791BDF84E
:10C690003F861A97111A1ABDF83F4FCE738C6F0060
:10C6A000088C73A226F87F00B37F00B4CC0C00FD89
:10C6B00072887F00B57F006A7F0076860AB7B59AD8
:10C6C000CC1770DDAF8639979F9797979497A5976A
:10C6D000A897A2867E97ABCCF8DEDDACCC0000DD5F
:10C6E0009ADD9C7F0077BDF5CA86FF978C979E7F69
:10C6F00000927F00B67F00937EC82C4F4B0D8EBFFB
:10C70000FF86FF979E860AB7B59A7F00817F008CCF
:10C71000BDF5CACEC6FB4FBDF44BCEC721FF738C0F
:10C72000CE0000FF7394FF738E863EBDF8DE4FCEC1
:10C73000B294BDF35B083CCEB294865CBDEDD226CC
:10C740001EBDE2CAFC721893522607FC721A93545B
:10C7500027033820D4865CBDEDD227037EF2AD18C6
:10C7600038DF5618BDEE57DC56DD4EBDEDE2DC522B
:10C770002634DC54261B8627BDEDD227AC7EC85B51
:10C7800045444954494E472044495341424C45444D
:10C790000D7D0092270DCEC7804FBDF44BBDF5CA6D
:10C7A0007EC7294D2A06CC00087EEEF60909098AC3
:10C7B00080ED00DF46DC4E9346E702DE4E09E700DF
:10C7C000BDF3C82705FF73AE201BFF73A6FF73AE32
:10C7D000FC73A2FD73A8BDF3ECFF73A4BDF53CFC94
:10C7E00073A6FD73A2DC4E9346C10526037EC729BE
:10C7F000FE73A2FF73AAF373AAFD73AC188CB28FF9
:10C800001823037EF352FD73A2BDF555FC73AEFDF4
:10C8100073A6DC4EFD73A8DC46FD73A4BDF53C7E1B
:10C82000C729CE01006F000926F8203AFEB5CD8C4D
:10C8300030392722B6C42E815326E7CE0142FF733A
:10C84000A4CE73D2FF73A6FC0140FD73A8BDF53CD6
:10C85000FC73A6FD73A27ECAAF0000CCC859FD735D
:10C860008CCCC441DD520908A600B1C42B27F8DFE7
:10C8700046A6003CDE52E6002B2811270B18C30009
:10C880000818DF5220F0DE4A08E600DF4A38083C8C
:10C89000E10027F2C180240838DE463CDE5220DD6C
:10C8A000DE4A08A60038363739BDF595BDF265DC9D
:10C8B00052FD7394B6C42C814F2709FC73948300F6
:10C8C00004FD7394CCC5ABDD527EC866BDE2CADC04
:10C8D00054FD7398DC52FD7396CCC5B5DD527EC80D
:10C8E00066BDE2CA7EC8F0CC0001DD545F4FDD5268
:10C8F000DC52FD739ADC54FD739CFC738CFD739EBB
:10C90000FF73A030200518C3000E18EC00271C1878
:10C91000BC73941826F0FF73AA18C3000EFD73AC05
:10C9200030FF73AEBDF555FE73AC35FE73A07EEDE2
:10C93000E9BDEDEF24037EF2ADFD73903CFE7394F0
:10C940002604387EF2ADBC7390270738BDF56E7EA5
:10C95000C93CEC02F3739CED02EC00F9739BB973D4
:10C960009A295BED00FC739A2B267D73962A066D3F
:10C97000002A4D20046D002B39EC0018BC7396255D
:10C9800031263D18EC0218BC739825262724203048
:10C990007D73962B066D002B2720046D002A13EC67
:10C9A0000018BC73962519260918EC0218BC739858
:10C9B000250E38FC739EFD738CFE73A02006ED00DF
:10C9C00038BDF56E7EEDE9BDE2CADC522605DC54C9
:10C9D0004D2A09CC00087EEEF67EF2AD3637862C65
:10C9E000BDEDD226F4BDE2CADC5226E7DC544D2B65
:10C9F000E23332DD48DC54934825D83CFE738CEC9E
:10CA000000847FDD502733189C48252E9C54270234
:10CA10002428BDF5CACECA204FBDF44B387EC6FED1
:10CA200043414E4E4F5420455241534520435552A9
:10CA300052454E54204C494E450DDE54DF52DE48DF
:10CA4000DF54CE73D2BDF3DA2404387EEDE9FF73F0
:10CA5000A6DC52C30001DD54BDF3DA2408FC73A642
:10CA6000FD73A22012FF73A4FE73A2FF73A8BDF58D
:10CA70003CFE73A6FF73A2DE5027CFDF54CE73D2E5
:10CA8000BDF3DA080808A600810D27BF813A27BB4D
:10CA900020F3BDEDE2810D2707813A27037EC9C748
:10CAA000CC73D2FD73A2BDF2A27EC6FEBDF2A286F9
:10CAB000FF2004BDF2A24F978C7F0081CE73D27FFE
:10CAC00000547F0055BDF3DA24037EC6FEFF738C4D
:10CAD00096B5271BBDF8DEEC00847FDD547F005245
:10CAE0007F005386019745BDF486863EBDF8DE087B
:10CAF0000808BDF5DBCCC479DD527EC866BDE2CA4C
:10CB00003CBDF2A2BDF3FF270738CC00157EEEF640
:10CB100032327ECACDBDEDEF24037ECBB23CFD7335
:10CB2000AA18EC00DD64EC02DD66CCEFC0DDAC38A9
:10CB30007F00547F0055862CBDEDD2260DBDEE57EB
:10CB4000DC522706CC00087EEEF6DC542BF6363796
:10CB500096442729862CBDEDD2270A862DB1C42EF6
:10CB6000BDEDD22613BDEE5796442711DC5226D4D4
:10CB7000DC542BD0DD5E200ACC00002003CC7FFFEC
:10CB8000DD5E3332DD543CBDF3C82512BDF517BD63
:10CB9000F3DA250AEC00847F935E27F025EEFE731E
:10CBA000AADC64ED00DC66ED02CCF8DEDDAC387E9C
:10CBB000C6FEBDEE57DC522706CC00087EEEF6DC42
:10CBC000542BF6363796442729862CBDEDD2270AFA
:10CBD000862DB1C42EBDEDD22613BDEE5796442747
:10CBE00011DC5226D4DC542BD0DD5E200ACC0000B0
:10CBF0002003CC7FFFDD5E3332DD5496763686012E
:10CC000097763CBDF3C82517BDF5177D0093262AFE
:10CC1000BDF3DA250AEC00847F935E27EB25E93823
:10CC20003284019776863BBDEDD2260BBDF8A181FB
:10CC30001327F9811127F57EC6FE383284019776D5
:10CC4000BDF83F7EC6FE863BBDEDD226037EEDE9F4
:10CC5000860DBDEDD2270C863ABDEDD227058D0A93
:10CC60007EEDE909BDF5CA7EEDE986019745BDF483
:10CC70005F27698623BDEDD22639C600A600813024
:10CC80002602C680D745BDE2CA9655847F9A45974D
:10CC9000458648C610A10027138642C602A1002778
:10CCA0000B8651C608A1002703C60A0908F7B59AE2
:10CCB0007ECCDCA600815C260A08BDE2CA96559DA2
:10CCC000AB2019867BBDEDD2260CBDCD01867DBD86
:10CCD000EDD226252006BDE2CABDF486862CBDED28
:10CCE000D2278B863BBDEDD2260139860DBDEDD214
:10CCF000270A863ABDEDD227037EF2ADBDF5CA09FB
:10CD000039BDE2CABDCF6ADC523637DC54363786CD
:10CD10002CBDEDD226E3BDE2CABDCF6A3332DD4879
:10CD20003332DD469352250E2706CC00167EEEF6F2
:10CD3000DC54934825F4BDCD50BDF02BBDCD509DA6
:10CD4000ABDC46935225EF2606DC54934824E739A2
:10CD50003CDE463CDE483CDE64DF46DE66DF4838CB
:10CD6000DF6638DF643839BDF595BDE2CABDF2A291
:10CD70003CBDF3FF270738CC00157EEEF618FE7396
:10CD80008C3CFE738E3C7F7394BF738E187ECACD2D
:10CD9000BDF2A2FC738E26037EF2ADBE738E38FF09
:10CDA000738E38FF738C38BDF56E7EEDE9FE738CA3
:10CDB0007F00547F0055BDF3EC7ECAC8BDE2CADCDB
:10CDC000522604DC5427037ECAF2BDF3F625037E07
:10CDD000CACD7EC6FEBE739238FF738C3838BDF55F
:10CDE000CA3CBDF45F2609BDEDEFDD542568202364
:10CDF0003CBDEDEFDD5424037EF2ADA600B1C42DA1
:10CE000097454FA70038BDF44B964509A700863AD1
:10CE1000BDF8DE3CFE738C3CCEFFFFFF738CBF730E
:10CE200092DC543736863ACEB394BDF35BCEB394DE
:10CE3000A600810D2606A7018630A700BDE2CABD67
:10CE4000EDE2810D268F380FDC54ED02DC52ED004F
:10CE50000E38FF738C3832B1C43132863BBDEDD20F
:10CE60002703BDF5CA862CBDEDD226037ECDE17E1B
:10CE7000EDE9A600810D270ABDF265862CBDEDD235
:10CE800027F67EEDE97EF2ADBDCF51862CBDEDD209
:10CE900026F3BDE2CA3CDE522609DE5427058C008B
:10CEA00009250738CC000B7EEEF618D7467F0047E1
:10CEB000D6474FC3E57518E600BDF6FD17BDEFC0B8
:10CEC0007C00479647914626E7202CBDCF518631FE
:10CED0009762862CBDEDD2261D8623BDEDD226316C
:10CEE000A600088132270B81342707813127037E72
:10CEF000F2AD976220DC3CFE73AAB6C42D814E27AA
:10CF000004DC422002DC66ED02DC64ED00387EEDDC
:10CF1000E9BDEDE28127270481222610CCEFC0DD98
:10CF2000ACBDCC6ACCF8DEDDAC7ECEF6BDE2CAD6B6
:10CF300062C134260C9652BDEFC09653BDEFC0209F
:10CF400004C13226059654BDEFC09655BDEFC020F2
:10CF500081BDEDEF2511FD73AA3CFE73AAEC00DD47
:10CF600064EC02DD6638397EF2ADCC0003DD46CCE0
:10CF70008000D39CDD48DC46D99B999A9352250BBF
:10CF80002608DC4893542503270139CC00167EEE91
:10CF9000F63CFC73A28373D22604387EEDE9188C2C
:10CFA0003EBF2534CECFAE4FBDF44B7EC6FE5052B1
:10CFB0004F4752414D20544F4F2042494720464F42
:10CFC0005220524F4D2028313633383220425954A6
:10CFD0004553204D4158290018C30142FD73D0CE5E
:10CFE000D2E74FBDF44BBDF5CACE17701ABDF86736
:10CFF000260D0926F7CED2F74FBDF44B7EC6FEBDF7
:10D00000F8A1811826037EC6FE8115268DCEB601B5
:10D01000DF5286019755FC73A2DD4ACC8D70DD4C42
:10D02000CE73D0BDD06038862BBDEDD23C260C4FE0
:10D030005FDD4CDD4ACEC000BDD0604FCED04BA6E8
:10D040000081242714BDD0E20820F43A303030307B
:10D050003030303030300D0A24BDD133387EEDE928
:10D06000DF4E7F00467C0046089C4A270696468194
:10D070001026F2863ABDD0E27F00479646BDD0C169
:10D08000DC4ED34C37BDD0C132BDD0C14FBDD0C1B5
:10D09000DE4EA600BDD0C1089C4A27107A00462665
:10D0A000F14F9047BDD0C1BDD0B620B44F9047BD21
:10D0B000D0C1BDD0B639860DBDD0E2860ABDD0E262
:10D0C00039369B47DD47323644444444BDD0D432E0
:10D0D000BDD0D439840F8B30813A25028B07BDD067
:10D0E000E2393CDE52A7008CB680270608DF5238B2
:10D0F000393CCEB601DF524F97548601BDF8DE961B
:10D1000055BDF8DE43BDF8DEA600BDF8DE9B5497A2
:10D1100054088CB68126F19654BDF8DEBDF8A18185
:10D120001527CF810626CB811826037EC6FE7C00FC
:10D13000553839DE528CB681270B6F00088CB681CA
:10D1400026F8BDD0F18604BDF8DEBDF8A181182710
:10D15000DA810626DE39BDE2CABDCF6ADC52DD6463
:10D16000DC54DD66862CBDEDD227037EF2ADBDE238
:10D17000CABDCF6ABDD2DC2406CC00167EEEF6B660
:10D18000C42E81532708DC529A40DA41DD5218DE62
:10D19000523CDE543C18862CBDEDD22707CC1770CC
:10D1A00036372020BDE2CADC522706CC00177EEEBF
:10D1B000F6DC543637862CBDEDD22608BDEDEF24C3
:10D1C000067EF2ADCC004EDD4E3332DD501838DF36
:10D1D0005438DF52183CDE4E8C004E260ACED2E781
:10D1E0004FBDF44BBDF5CABDD2002620DE4E8C00EB
:10D1F0004E260ACED2F74FBDF44BBDF5CA7ED2CE35
:10D20000DE501ABDF86726030926F739BDF8A1815B
:10D210001826037ED2CE811526CD8601974720346D
:10D220007C0047BDD200260D3338BDD2DC24037EFE
:10D23000D2AE7ED2CEBDF8A1333881062716811832
:10D2400026037ED2CE811527043C3720D6DF66D751
:10D25000657A0047BDD2DC254BDE663CD665377F5C
:10D26000005A7F005B8601BDF8DE9647BDF8DE43BD
:10D27000BDF8DEBDD2DC2515965A8180271EBDF093
:10D280002BBDF8DE9B5B975B7C005A20E6965A81AB
:10D290008027094FBDF8DE7C005A20F1965BBDF86F
:10D2A000DE7ED2208604BDF8DEBDD20026197300D2
:10D2B00064730065DC664353C30001DD66DC64C94A
:10D2C000008900DD642007BDF8A1810626D6DE4E68
:10D2D000DC64ED00DC66ED02387EEDE99653906586
:10D2E0002604DC5493663957414954494E47204639
:10D2F0004F52204E414B004E414B204E4F54204642
:10D300004F554E44204245464F52452054494D45C5
:10D310004F555400BDE2CADC522706CC00187EEE01
:10D32000F6DC54260D96431A914327FB4FDD6C7EA5
:10D33000EDE9DD6E200108A600B1C43127F8813A7D
:10D34000272C810D27283C20091ADC6C936E270BB3
:10D3500024097B401527F2387ECAF2DD6C38CC00F8
:10D3600000DD54BDF3F625037ECACD7EC6FE3C1A11
:10D37000DC6E936C270925022AF5862ABDF8DECEDD
:10D380000000DF6C387EEDE99DA53838CC000C7EBE
:10D39000EEF6BDE2CADC52270DCC000C7EEEF63C68
:10D3A0008DE6387EEDE9DC544D26F4C10E24F0C143
:10D3B00008241786805D2704445A20F9369A159769
:10D3C00015329A8B9720978B201EC00886805D2788
:10D3D00004445A20F9B1C43124024444369A0397D4
:10D3E00003329A8A9701978A862CBDEDD227A37EB5
:10D3F000EDE99DA83838CC000C7EEEF6BDE2CADC23
:10D4000052270DCC000C7EEEF63C8DE6387EEDE921
:10D41000DC544D26F4C10E24F0C108241886805D2A
:10D420002704445A20F9364394159715329A8B975E
:10D4300020978B2021C00886805D2704445A20F95C
:10D44000B1C43124024444364394039703329A8A88
:10D450009701978AC00E862CBDEDD2279F7EEDE9FD
:10D46000BDD5D986809A8A9701978ABDEDE281223F
:10D47000270481272610CCD4BCDDACBDCC6ACCF807
:10D48000DEDDAC7EEDE9BDD619DC7B2604DC792738
:10D490001BBDF02BBDD4BCDC7B830001DD7BDC79C4
:10D4A000C2008200DD7926E9DC7B26E53CFE73AA1A
:10D4B000DC64ED00DC66ED02387EEDE93CDE7D8C5F
:10D4C000011324010FBDD5D3717F03BDD5D3C60889
:10D4D000442505717F0320057280032000BDD5D34C
:10D4E0005A26ED728003380E39BDD5D9BDD61986BE
:10D4F0002CBDEDD227037EF2ADBDE2CADC7B260750
:10D50000DC7926037ED4AC86FE948B9720978B869D
:10D510007EB7010CCCD57AFD010DDC522706CC007C
:10D52000257EEEF60FDC42D354DD54DC40D953990E
:10D5300052DD5296AE8900974E7F007FDF467F0016
:10D5400080DC7D83011325037A00800E01010F72B8
:10D5500001140E1A0F967F2616964E90AE251026B1
:10D56000EADC529340250826E2DC54934224DC7125
:10D57000FE140E86FF97807ED4AC71FE1496802731
:10D58000010ED61737C4F7D717DC7D04D37D18BD3D
:10D59000D5D5C68096150425070101BDD5D320F445
:10D5A00017DE46BDEFC0DC7B830001DD7BDC79C28A
:10D5B000008200DD79DC7D04047B011526058300F3
:10D5C0000126F6DC792608DC7B260486FF977F336C
:10D5D000D7173BDE7D0926FD39BDE2CA3CDC52DDB2
:10D5E00046DC54DD48BDEF75CC04B0DD53BDF06DB5
:10D5F000DC52260CDE548C0FA024058C001E240A5D
:10D6000038CC00197EEEF67EF2AD18830007DD7D82
:10D6100038862CBDEDD226EF39BDE2CADC52DD7969
:10D62000DC54DD7B862CBDEDD226DCBDEDEF25D7AD
:10D63000FD73AA3C18EC00DD64EC02DD663839BDF0
:10D64000E2CABDF2A23CBDF3FF270A387F0081CCBD
:10D6500000157EEEF6DF823886FF97817EEDE9BD0C
:10D66000CF51860DB773AC862CBDEDD22616865CE5
:10D67000BDEDD22636BDE2CA9655B773AC862CBD39
:10D68000EDD227273C4FCEB394F673ACBDF35DCEFD
:10D69000B394A600B173AC270C08DF5238BDEFC0BD
:10D6A0003CDE5220EDBDEFC07ECEF7BDE2CADC52BB
:10D6B0002706CC001A7EEEF6DC54272ADC54DD5215
:10D6C000BDF867270FBDF8A136BDEFC032B173AC0E
:10D6D000271120EC1ABDF86726E2DC52830001DD39
:10D6E0005226F17ECEF6BDF86727F8BDF8A1BDEF52
:10D6F000C020F0BDCF51860DB773AC862CBDEDD2E6
:10D700002612865CBDEDD227037EF2ADBDE2CA963D
:10D7100055B773AC3CBDF02BB173AC2705BDF5CC50
:10D7200020F33836863BBDEDD232270C810D26051D
:10D73000BDF5CA2003BDF8DE7ECEF6BDF2A2CCB2A6
:10D740008FB373A2DD547F00527F00538606974546
:10D75000BDF4867EC6FEBDE2CADC522706CC001BA5
:10D760007EEEF6DC54188C00DC1825F13637862C5A
:10D77000BDEDD226E8BDE2CADC5226E1DC54260427
:10D780003232203505DD5425D43332DD463C867EE9
:10D79000B70106CCD7BCFD010771FD039608DC0973
:10D7A000D346DD0B8601970F860897081ADC4626BC
:10D7B000FB7F00088600970F387EEDE99608DE545F
:10D7C000270E09DF5488019708DC0BD346DD0B3B9D
:10D7D000DC0BD346DD0BDF463B86FF3620024F369F
:10D7E000BDF2A23297927EC6FEBDE2CADC52270687
:10D7F000CC001C7EEEF6DC542706DDAF860120014E
:10D800004F97767EEDE9A600812D260DBDF86C269A
:10D81000FB86FF0897777EEDE9812B27037EF2AD2B
:10D820004F20F0B673B0BA73B1BA73B4BA73B5BA65
:10D8300073B8BA73B9BA73BCBA73BDBA73BEF673B0
:10D84000BF271FC12025028AFFBA73C0BA73C1BAAD
:10D8500073C2F673C3270BBA73C4BA73C5BA73BE67
:10D860002706CC00267EEEF67F004A7F004BFC7335
:10D87000B2DD4CCC003CDD484F5FDD46DD52FC7331
:10D88000B6DD54BDF1A1BDD95E4F5FDD46DD52CCA2
:10D890000E10DD54FC73BADD48BDF1A1BDD95E4F59
:10D8A0005FDD465CDD52F673BF5ADD48CC5180DD4A
:10D8B00054F673C7C1292404CB142008C050251581
:10D8C000C1142411D75E54545C4FD348DD48F6731D
:10D8D000C3C10D2506CC001D7EEEF6D7463CCED941
:10D8E0006DC1032409D65EC40326037A00495F7A1A
:10D8F00000462707EB0089000820F438D348DD48AC
:10D90000BDF1A1BDD95E4F5FDD52D65EDD54CC01C5
:10D91000E1DD46CC3380DD48BDF1A1BDD95EBDED72
:10D92000EF250E3C18DC4AED00DC4CED02387EEDB4
:10D93000E9DC4CDD484FD64BDD465FDD52C664DD89
:10D9400054BDF1A10FDC50DD42D64FD7418664D6DD
:10D950004A3DDB4E8900D74097AE0E7EEDE9DC50A4
:10D96000D34CDD4CDC4ED94B994ADD4A391F1C1F84
:10D970001E1F1E1F1F1E1F1E1FBDEDEF3C24460F46
:10D9800096AE9752DC40DD53DC4297550ED75ECC05
:10D990000064DD485FDD46BDF06DDC53DD5F96550C
:10D9A00097619651D65EDD544F5FDD52DD46C66409
:10D9B000DD48BDF06DDC549B61DD54DC5FC900893E
:10D9C00000DD52200918EC02DD54EC00DD52188C09
:10D9D0008000250738CC001E7EEEF6CC0001DD4627
:10D9E000CC5180DD48BDF06DDE543CDC4EDD52DCB8
:10D9F00050DD544F5FDD46CC0E10DD48BDF06DDCD0
:10DA000054FD73BA5FFD73B8DC4EDD52DC50DD545B
:10DA10004F5FDD46CC003CDD48BDF06DDC54FD734E
:10DA2000B65FFD73B4DC50FD73B25FFD73B03818A0
:10DA30007F00527A00527C0052BDDAA2260A83018E
:10DA40006E24F3C3016E200883016D24E9C3016DC8
:10DA50003637D652CB50C1642502C0644FFD73C621
:10DA60005FFD73C43332CED96D7F00547F00537C89
:10DA7000005337E600BDDAA2260937D653C1023378
:10DA800026015C08D75533935424E4D3544F5CFDEE
:10DA900073BED653FD73C25FFD73BCFD73C0387E89
:10DAA000EDE936965284033239CC00207EEEF67EC4
:10DAB000F2ADBDEDE28122270481272613BDDB6193
:10DAC000CCDB44DDACBDCC6ACCF8DEDDAC7EEDE970
:10DAD000BDE2CA18DE523CDE543C18862CBDEDD2A5
:10DAE00026CDBDE2CADC5226C0965426BCD65527A8
:10DAF00050C12124B4BDDB61D7461838DF5438DF6C
:10DB00005218D64686209046270F78005579005443
:10DB10007900537900524A20EF7B80522705720426
:10DB200003200371FB0372041571FB15780055790E
:10DB300000547900537900525A26DE72201571DFA5
:10DB4000157EEDE9C608492405720403200371FB24
:10DB50000372041571FB155A26EC72201571DF153E
:10DB60003986049A8A9701978A86249A8B972097F8
:10DB70008B71DB15398627BDEDD2270A8622BDEDD4
:10DB8000D227037EF2ADBDDBB1974EBDDBB136BD12
:10DB9000DBB11632DD46BDDBB1BDDBB1D64E270EA3
:10DBA0005AD74E3CDE46A70008DF463820EB7EED14
:10DBB000E98D0A48484848368D03331B39A60008CA
:10DBC0008030250C810A250B800725048110250350
:10DBD0007EF2AD39CC00217EEEF67EF2ADBDE2CA1A
:10DBE000DC5226F0DC54183C18862CBDEDD226EA17
:10DBF000BDEDE28122270481272610183818DDACFC
:10DC0000BDCC6ACCF8DEDDAC7EEDE9BDE2CA18DE43
:10DC1000523CDE543C18862CBDEDD22705CC004E7C
:10DC20002005BDEDEF25B3FD73AA1838DF5438DFAA
:10DC30005238DF46183CBDF86C26FBCEDC473CDE94
:10DC4000463CDC54DE52393CFE73AAED021838180B
:10DC5000ED00387EEDE97EF2AD38CC00247EEEF6A4
:10DC6000BDEDEF25F13C188C719C25EDEC00DD56E7
:10DC7000EC02DD54188372184353C3000154173665
:10DC8000BDF69ADC54DD56324CBDF69A387EEDE98D
:10DC90007EF2AD38CC00247EEEF6BDEDEF25F13CF2
:10DCA000188C719C25ED3C188372184050C30001FC
:10DCB000541736BDF64ADC56DD52324CBDF64A38B2
:10DCC000DC56ED02DC52ED00387EEDE9BDE516DCF8
:10DCD000522615DC54188C0014250C8C0C012407DA
:10DCE00018FD72887EEDE918CC00237EEEF67F00E9
:10DCF000B37F00B4867BBDEDD2260EBDEDEF250CC3
:10DD0000DDB3867DBDEDD226037EEDE97EF2AD7FEB
:10DD10000008BDEDEF251CFDB598867EB70109CC46
:10DD2000DD36FD010AC602D708D608DC0DDC09C6BF
:10DD300012D7087EEDE99608FEB598EC02C3000103
:10DD4000ED02EC00C9008900ED00DE0D3B86FF9777
:10DD50004F860197503CCC0052FD73ACBDEDEF25D2
:10DD6000123637862CBDEDD226073332FD73AC2038
:10DD700002323338BDE2CADC52DD64DC54DD668633
:10DD80002CBDEDD227037EF2ADBDEDEF25F8FD737E
:10DD9000AA3C96B636861897B6BDF83FCE00649674
:10DDA000431A914327F9BDF86726EE0926F1861537
:10DDB000BDF8DE7C004FD64FC11426208618BDF872
:10DDC000DEFE73AA4FED025FED00FE73ACDC66ED84
:10DDD00002DC64ED003297B6387EEDE9BDDE6127E6
:10DDE000CDBDF8A181182604C61520D581042609C9
:10DDF0008606BDF8DED64F20C88101269CBDDE0C0C
:10DE000026978606BDF8DE7C005020D0CEB394C69F
:10DE100083BDDE51A700085A26F7FCB3945311279F
:10DE20000139CEB3964FAB00088CB41626F8B1B4C6
:10DE300016270139B6B3944C915026064A915027C3
:10DE40000139CEB396A600BDEFC0088CB41626F5F6
:10DE5000393CBDDE61382704BDF8A13938387EDD94
:10DE600099CE01F4BDF86727013996431A914327EB
:10DE7000F90926F03938CC00017EEEF67EF2ADBD10
:10DE8000EDEF240ABDEE57964427F1CC0052FD7306
:10DE9000AA3C18EC0026DEEC02FD73AC38862CBDE3
:10DEA000EDD226D87EDEBB863BBDEDD227F63CFE0A
:10DEB00073AAFC73ACED02387EEDE9CCE0E8DD46F8
:10DEC000BDEDE2DF483CDE46A100260908DF46380A
:10DED00008A60020F0A6002B1908A6002AFB0808B7
:10DEE000A6002604387EF2ADDF4638DE48A6007E66
:10DEF000DEC53C16584FC3E0D218EC00186E00384F
:10DF0000A601BDE0C6387EDEA738A601BDE0C63852
:10DF1000BDE2CADC5227037EEEF6DC5427188300EC
:10DF200001B373AC4D2606C18024EC200881FF2686
:10DF3000E6C18025E217BDE0C67EDEA738A601381F
:10DF4000E600C1412706C14226058B100820E736AE
:10DF5000BDE2CABDE08D270C328B30BDE0C6BDE00E
:10DF6000A77EDEA732BBC431BDE0C6BDE0B27EDE17
:10DF7000A738A6013836BDE2CADC5227037EEEF68A
:10DF8000DC544D26F837862CBDEDD227037EF2AD4A
:10DF9000BDE2CADC5226E6DC544D26E1BDE08D260A
:10DFA00016DF46183332BDE0C617BDE0C61817BDF0
:10DFB000E0C6DE467EDEA7DF461833328B107EDFFA
:10DFC000A638A601387EDF4F38A60138E600C141E9
:10DFD0002709C14227037EF2AD8B4036088623BD58
:10DFE000EDD2262EBDE2CA32BDE0C6BDE0B27EDE75
:10DFF000A738A6013836B6C42D802BBDEDD2261227
:10E00000BDE2CA32BDE0C6BDE0A77EDEA738A601EC
:10E010003836BDE2CABDE08D260C328B20BDE0C68D
:10E02000BDE0B27EDEA79654270C328B30BDE0C631
:10E03000BDE0A77EDEA7328B1020E238A601BDE04E
:10E04000C638BDE2CABDE0B27EDEA738388622BD42
:10E05000EDD22604167EE0608627A100260D160864
:10E06000A6000811270BBDE0C620F5BDE2CABDE041
:10E07000B2862CBDEDD227D57EDEA73838BDE2CAE8
:10E08000BDE0A7862CBDEDD227F37EDEA7A600B1AA
:10E09000C42B26030820F6812C260B08A600088135
:10E0A0005827037EF2AD39DC52260E9654BDE0C6E9
:10E0B000200EDC522706CC00277EEEF6965426F979
:10E0C0009655BDE0C6393CFE73ACA70008FF73ACA3
:10E0D0003839DEFFDF09DF3CDF71DFC1DFC8DFF188
:10E0E000E00DE03BE04BE07B4E4F5080014C535243
:10E0F00044800441534C44800554415080065450A0
:10E10000418007494E5880084445588009434C5681
:10E11000800A534556800B434C43800C5345438043
:10E120000D434C49800E534549800F5342418010A6
:10E130004342418011544142801654424180175855
:10E1400047445880184441418019534C50801A412B
:10E150004241801B5453588030494E5380315055B2
:10E160004C41803250554C428033444553803454A6
:10E170005853803550534841803650534842803779
:10E1800050554C5880385254538039414258803A47
:10E19000525449803B50534858803C4D554C803D2B
:10E1A000574149803E535749803F42524181204266
:10E1B000524E81214248498122424C53812342439D
:10E1C0004381244243538125424E45812642455195
:10E1D00081274256438128425653812942504C811F
:10E1E0002A424D49812B424745812C424C54812D76
:10E1F000424754812E424C45812F4E454782404331
:10E200004F4D82434C53528244524F5282464153A7
:10E2100052824741534C8248524F4C8249444543B5
:10E22000824A494E43824C545354824D434C52824D
:10E230004F41494D83614F494D836245494D836547
:10E2400054494D836B4A4D50844E53554244868306
:10E250004144444486C3435058868C4C444486CC45
:10E260004C4453868E4C445886CE53554285804349
:10E270004D5085815342438582414E4485844249B5
:10E280005485854C44418586454F52858841444399
:10E2900085894F5241858A414444858B535441417D
:10E2A00087875354414287C7535453878F4A5352E9
:10E2B000878D53544487CD53545887CF4253528847
:10E2C0008D4442890044578A0000BDE2FAF6C43109
:10E2D000A600081127FA817C27020939DC54373659
:10E2E000DC523736BDE2FA32339A52DA53DD52321B
:10E2F000339A54DA55DD547EE2CDBDE32AF6C42BC1
:10E30000A600081127FA812627020939DC5437367E
:10E31000DC523736BDE32A32339452D453DD5232C5
:10E32000339454D455DD547EE2FDBDE3D0A60008FD
:10E33000B1C43A27F809813C2504813F250139DC25
:10E34000543736DC523736CCC649DD527EC866BDFE
:10E35000E395250B860197552008BDE39526F57FAB
:10E3600000557F00547F00537F005239BDE395274D
:10E37000EE25EC20DFBDE39527DA25D820E1BDE3CB
:10E380009526DC20CFBDE39524D520C83233DD525D
:10E390003233DD5439DF4E381838DF5038183C1826
:10E3A0003CDE503CDE4EBDE3D03233DD463233DD61
:10E3B0004896469852182A0CDE529C462610DE5487
:10E3C0009C481839DE469C522604DE489C54183975
:10E3D000862DBDEDD22606BDEF757EE429862BBDC8
:10E3E000EDD2BDE43A862BBDEDD22635DC5437366E
:10E3F000DC523736BDE43A3233DD463233DD48DCB9
:10E4000054D348DD54DC52974ED9479946DD529695
:10E410004E98462BD0964E98522ACACC00097EEED2
:10E42000F6862DBDEDD2270139DC543736DC523764
:10E4300036BDE43ABDEF5D7EE3F7BDE4CE862ABD8E
:10E44000EDD22621DC523637DC543637BDE4CE33EC
:10E4500032DD483332DD46BDF14BDC4EDD52DC505F
:10E46000DD547EE43DA600812F2705812527013953
:10E470003C087F00447D00522A067C0044BDEF5DCD
:10E48000DC523637DC543637964436BDE4CE32970C
:10E49000447D00522A067A0044BDEF5DDC52DD4621
:10E4A000DC54DD483332DD543332DD523CBDF06D97
:10E4B00038183836A60081252608DE4EDF52DE5099
:10E4C000DF54321896442703BDEF5D7EE43D090812
:10E4D000A600812027F981302504813A2530812842
:10E4E000273E81262728A6018141250C815B24082F
:10E4F000CCC5BFDD527EC866BDEDEFDD52251E3CAA
:10E500000FDE52EC00DD52EC020EDD543839BDEE68
:10E510005796442708398628BDEDD227047EF2ADF0
:10E5200008BDE2CA8629BDEDD226F239BDE51696B0
:10E53000522A03BDEF5D96522B0139CC000A7EEEC4
:10E54000F6BDE516DC522706CC000B7EEEF63C8DC0
:10E550000738DD545FDD5239DE548C0008250A9DF2
:10E560009F3838CC000B7EEEF618C3E57518E60030
:10E57000BDF6FD4F391F1B1E1A1D191C1818FE73FE
:10E58000AA3CDE643CDE663C188628BDEDD2262916
:10E59000BDCF517F00527F00537F0054862CBDEDCC
:10E5A000D226288623BDEDD2260FA6000881342767
:10E5B0000B81322711813127127EF2ADBDF02B97EE
:10E5C00052BDF02B9753BDF02B9754BDF02B9755B0
:10E5D0003CFE73AADC66ED02DC64ED00381838DF1F
:10E5E0006638DF6438FF73AA188629BDEDD226C9C4
:10E5F000399DA23838CC000C7EEEF68628BDEDD2CF
:10E600002657BDEF75DC54053736BDE2CADC52270C
:10E610000CCC000C7EEEF63C8DD7382021DC544D1E
:10E6200026F5C10E24F1C108243386805D270444F9
:10E630005A20F93643948B9720978B3294152707ED
:10E640003233C3000120023233DD54862CBDEDD2BB
:10E6500027B38629BDEDD227037EF2AD39C00886E7
:10E66000805D2704445A20F9B1C43A240244443658
:10E6700043948A9701978A32940320C2BDE5169687
:10E68000522A06CC000D7EEEF6CC0000DD46DD48B9
:10E69000DD4EDD50DD4CCC4000DD4A860F975ADC64
:10E6A00048D350DD58DC46D94F994EDD56DC58D35F
:10E6B0004CDD58DC56D94B994ADD5674004E760035
:10E6C0004F760050760051DC529356251E2606DC0C
:10E6D0005493582516DC56DD46DC58DD48DC50D313
:10E6E0004CDD50DC4ED94B994ADD4E74004A760021
:10E6F0004B76004C76004D74004A76004B76004C09
:10E7000076004D7D005A2609DC4EDD52DC50DD548A
:10E71000397A005A20893CBDEF75C61CBDF6FDD77D
:10E72000547F00467F0047CC028DDD48BDF06D3838
:10E7300039BDE516DC522706CC000E7EEEF6DC5421
:10E740004D26F517C4FC105497464FC3E7703C188C
:10E75000EC00DD4EA30296463DCB0204044353C3B6
:10E760000001D34EDD542A0673005273005338392A
:10E7700005DC05DC055A04AB043603DF038E0353C6
:10E78000032102F402CD02A90288026A024E02337A
:10E79000021A020301EC01D701C201AE019B0189FB
:10E7A0000176016501540143013201220112010287
:10E7B00000F200E200D300C400B400A4009500857C
:10E7C0000076006600560046003500240013000164
:10E7D000FFEEFFDCFFC8FFB3FF9DFF86FF6DFF5319
:10E7E000FF35FF15FEF0FEC4FE8FFE48FE1BFE1B2C
:10E7F000FE1BBDE5163C7D00522A09DC545343C381
:10E800008001DD54DC54847FDD52188C40001825D3
:10E8100005CC80009352DD46164F05C3E8C718ECBF
:10E8200000DD48EC02A300974E96473D97517F00CC
:10E8300050D64E96473DD350D3487F00527F005369
:10E840007D00542A154353730052730053C30001D3
:10E8500018DC52C9008900DD5218DD543839BDE595
:10E86000163C7F00567D00522A06BDEF5D7A0056A9
:10E87000DC52270738CC000F7EEEF6DC5427462BFF
:10E88000F3CEE8C77F0057EC00189C541824070803
:10E89000087C005720F1DD4A0909EC00DD4CDC4A18
:10E8A000934CDD48CE0000DF46DC54934CDD537FB3
:10E8B0000055BDF06D96574A5FD354DD547D005628
:10E8C0002703BDEF5D3839000003240648096A0CB0
:10E8D0008C0FAB12C815E218F91C0B1F1A22232546
:10E8E0002828262B1F2E1030FB33DE36BA398C3CFD
:10E8F000563F1741CE447A471C49B44C3F4EBF5156
:10E9000033539A55F558425A825CB35ED760EB6236
:10E91000F164E866CF68A66A6D6C236DC96F5E709E
:10E92000E2725473B575047641776B788479897A8D
:10E930007C7B5C7C297CE37D897E1D7E9C7F097FBE
:10E94000617FA67FD87FF57FFFCC0002DD545FDDBD
:10E950005239FCFFE8DD547F00527F0053393CCE32
:10E96000C403BDEE573839CC00107EEEF6BDE51677
:10E97000DC5226F3965426EFD655BDEF755D27E79A
:10E98000C12124E386BF948A9701978A968B8A14C3
:10E99000978B972071EB157210152012780055791E
:10E9A000005479005379005272041571FB157B40B5
:10E9B0000327037C00555A26E339CC00117EEEF67E
:10E9C000BDE516DC5226F3DC5427403C18968A84B9
:10E9D000FE9701978A867EB70109CCEA0CFD010AF1
:10E9E0007F00547F005596431A914327FB01010194
:10E9F00001D608DC0D9643C6120FD7080E1A9143B4
:10EA000027F796430926F27F00083839960884EFE5
:10EA10009708DC0DDC54C30001DD54DC52C90089C9
:10EA200000DD523B9608DE4A08DF4A84E29708DEA2
:10EA30000DDF54B4C42B270EDE548C80002407DE77
:10EA40005208DF52DC093B960820F47EF2ADCC0080
:10EA5000127EEEF68628BDEDD226F0BDE2CADC526B
:10EA600026ECDC5427E8183C18862CBDEDD226DBBA
:10EA7000BDE2CADC5226D7DC5427D3DD4E18381845
:10EA8000DD508629BDEDD226C23C968A84FE9701D0
:10EA9000978A867EB70109CCEA24FD010A867EB7F3
:10EAA0000103CCEA47FD01047F004A7F004B7F0051
:10EAB0004CC602D708CC0000DC09D608DC0DDC0906
:10EAC0009643C6160FD7080E1A914327099643DEC0
:10EAD0004E092731DF4E0FDE4A092611964C260DCE
:10EAE0007C004CDE52DF46DE54DF4820D79C5026A7
:10EAF000D30E7F0008DC549348DD54DC52D2479299
:10EB000046DD5238397F0008CC0000DD52DD543834
:10EB100039BDE5167F005ADC522A06CC00137EEE82
:10EB2000F63C271574005276005376005476005553
:10EB30007C005ADC5226ED2011DC5427DE2B0B78AA
:10EB400000557900547A005A20EF7F00467F004735
:10EB5000DC54C3B172DD487C0047CCB172DD52CCCD
:10EB600017ADDD54BDF06DDC54DD567F0058DC4F31
:10EB7000DD52965197547F0055BDF06DDC54D3574C
:10EB8000DD57965689009756965680809756DC58E2
:10EB900005DD58DC565949DD56730056DC574353A2
:10EBA000C30001DD57965689009756CE0000DC560B
:10EBB000DD54DD482A03CEFFFFDF52DF46BDF14BB7
:10EBC000DC4EDD5EDD54CC994BDD48CC0000DD46EB
:10EBD000DD52BDF14BDC4EC3F622DD54DC5EDD4878
:10EBE000CC0000DD52DD46BDF14BDC4EC3E2A8DDBA
:10EBF00060CC0002DD5EDC57DD544FD6562A02861B
:10EC0000FFDD52DC54363705DD58DC5236375949C2
:10EC1000DD56CC0000DD46974896609749BDF14B24
:10EC2000DC4FD358DD58DC56C9008900DD564FD67D
:10EC30004E2A0286FFD356DD56D661D7493332DDE0
:10EC4000523332DD54BDF14BDC4ED358DD58DC5627
:10EC5000C9008900DD564F5F7D004E2A03CCFFFFBF
:10EC6000D356DD56DC5783875DDD53965682009779
:10EC7000524F965A9B529752DC53DD5436374FD63B
:10EC8000522A0286FF3637DD5286B19749CC000002
:10EC9000DD469748BDF14BDC4EDD56DC50DD58C6F5
:10ECA00072D7493332DD523332DD54BDF14BDC4E85
:10ECB000D357DD548600D6562A0286FFC900890044
:10ECC0007D004E2A03C3FFFFDD523839BDE516DC57
:10ECD000522B0B83000A2506CC00147EEEF6DC5284
:10ECE000DD56DC54DD58DC53DD5496529753CC008E
:10ECF00001DD46CC62E4DD48BDF14BD64E2A0CC1A5
:10ED0000F02408CC0000DD52DD54394F5CD75A2A7C
:10ED10000286FFDD5416DD52CCB172DD487F00461D
:10ED20007F0047BDF14BDC509358DD54DC4ED25789
:10ED30009256DD52DC524756DD5EDC544656DD60AD
:10ED40008607975B3CCCFFFFDD52CCFFF3DD54CE52
:10ED5000EDB6BDED827A005B26F8965A2B13270F8D
:10ED60007800557900547900537900524A26F138D9
:10ED7000397700527600537600547600554C26F1D0
:10ED80003839DC5EDD46DC60DD48BDF14B9650482D
:10ED9000DC4E5949DD54CC00007D004E2A03CCFFE7
:10EDA000FFDD52EC02D354DD54EC00D9539952DD0F
:10EDB0005208080808390000005BFFFFFDDE000074
:10EDC0000AABFFFFD55500008000FFFF00000001E7
:10EDD0000000160908A600812027F908112701095B
:10EDE0003908A600812027F939BDF2887EF2AD09E5
:10EDF00008A600812027F9813F262608A600812049
:10EE000027F981282705CC00400C39BDE516DC52D6
:10EE10002627DC544D2622C106241E0505C373B0E7
:10EE2000398040240139262008BDE516DC52260928
:10EE3000DC5418BC7288182506CC00027EEEF6055C
:10EE4000054353C372190C39811B25020D3908483B
:10EE500048164FC3721839BDEF757F0044BDEDE20F
:10EE60007F0046812626037EEF17813024013981F9
:10EE70003A250139840F7D0044260A7C00449755C9
:10EE800008A60020E57C0044D644C1052414974719
:10EE9000DC5405DD540505D354D346DD5408A600E3
:10EEA00020C89747DC5405DD54DD50DC5259492B0E
:10EEB00042DD52DD4E78005179005079004F7900E3
:10EEC0004E2B3078005179005079004F79004E2B4D
:10EED00022DC54D350DD54DC52D94F994E2B14DD33
:10EEE00052DC54D346DD54DC52C90089002B04DDCA
:10EEF0005220AACC00033CCEEEFD7EF2B3484F5721
:10EF00003F20204552524F52202300574841543F42
:10EF10000D534F5252590D08A6008148270909394F
:10EF20009644260209093908A600803025F2810A94
:10EF3000250A8007810A25E8811024E47C0044D654
:10EF400044C10924AEC604780055790054790053B1
:10EF50007900525A26F19B5597557EEF2773005240
:10EF6000730053DC544353C30001DD54DC52C90029
:10EF70008900DD52397F00527F00537F00547F00AB
:10EF800055393CFE738C3CCEEFAAFF738CBDEFC0AD
:10EF900038FF738C38393CFE738C3CCEEFAAFF737C
:10EFA0008CBDF02B38FF738C38390001004441547C
:10EFB0004146494C45204F56455252414E47450027
:10EFC0003CBDEFC63839367D00642609DC65052571
:10EFD000048107250B329D943838CC00047EEEF670
:10EFE000331807360F1837D617C4F81B4C330F30B9
:10EFF0008C010125059F688E00FF971737DC66841A
:10F000007FC340001832A700D617C4F8D717308C3A
:10F01000010026029E6816320637DC66C30001DD59
:10F0200066DC64C9008900DD6432393CBDF03138EA
:10F03000397D00642609DC650525048107250A9DC4
:10F04000973838CC00057EEEF616073617D617C46B
:10F05000F81B4C0F308C010125059F688E00FF972F
:10F0600017DC66847FC3400018A600209BDE46267E
:10F070004BDE4826083838CC00067EEEF6DE5226F7
:10F080003BDC54CE00007C005278004979004824D3
:10F09000F576004876004993482404D348200108B7
:10F0A0007A0052270B18051874004876004920E7AB
:10F0B000DF54CE0000DF52DF4EDD50397F004ADEE4
:10F0C00052DF4EDE54DF50CE0000DF52DF547C00B2
:10F0D0004A78004979004879004779004624EF765C
:10F0E0000046760047760048760049DC509348DDBC
:10F0F00050DC4ED2479246DD4E2410DC50D348DD22
:10F1000050DC4ED9479946DD4E20127C0055240D27
:10F110007C005424087C005324037C00527A004A6B
:10F12000271A7800557900547900537900527400F9
:10F130004676004776004876004920AF393CCE003D
:10F140004686106F00084A24FA38397F00447D0053
:10F15000522A067C0044BDEF5D7D00462A1A7A00E3
:10F1600044730046730047DC484353C30001DD4845
:10F17000DC46C9008900DD46BDF1A1964E2A06CCC9
:10F1800000077EEEF69644271773004E73004FDC9F
:10F19000504353C30001DD50DC4EC9008900DD4EF1
:10F1A000397F004E7F004F9649D6553DDD50D655EC
:10F1B000272F9648270B3DD34FDD4F964E8900975A
:10F1C0004ED6559647270A3DD34EDD4E24037EF298
:10F1D0005FD6559646270A3D4D26F3DB4E25EFD7E1
:10F1E0004ED65427389649270B3DD34FDD4F964EC8
:10F1F0008900974ED654964827083D4DD34E25CECC
:10F20000DD4EF6C42FC1452614D6549647270A3D35
:10F210004D26BBDB4E25B7D74E964626B1D6532793
:10F2200023964927093DD34EDD4E2533974ED653BD
:10F230009648270A3D4D2627DB4E2523D74E964775
:10F240009A46261BD65227169649270A3D4D260F69
:10F25000DB4E250BD74E96489A479A46260139CC65
:10F2600000077EEEF6BDEDEF25433736863DBDED5A
:10F27000D2263ABDE2CADF46380FDC52ED00DC543C
:10F28000ED020EDF52DE4639863ABDEDD22605325A
:10F29000327ECAF5860DBDEDD226063232087ECA10
:10F2A000BF39BDEDE2810D27F8813A27F43C4F5F6D
:10F2B000CEEF0B0EDD547F00527F0053CCF8DEDD25
:10F2C000AC7F00B57D008127273CFE738C8CFFFF4F
:10F2D00038271D96B681182606BDF8DE7F00B68E4B
:10F2E000BFFFCC0000FD738EFD7394DE82BDCACDDE
:10F2F0007F00B37F00B496B6270CBDF8DE96B681CA
:10F300001826037F00B64FBDF44B860AB7B59ADCCA
:10F310005427097F0045BDF486BDF5CAFE738C8C69
:10F32000FFFF26037ECDD5EC0026037EC6FEBDF58D
:10F3300020183809DF4618A600810D270FBDF5CC2F
:10F340009C462605863FBDF5CC0820EBBDF5CC7E5E
:10F35000C6FE3CCEEF114F5F7EF2B3C60DD74636E8
:10F36000DF5218C300F0DD54DE52BDF8A1817F27C3
:10F37000418108273D810A27F1810027ED8103267D
:10F38000113337C13A260B33383838FF738C387E47
:10F39000F5EDA700089146261233C13A270CBDF8B7
:10F3A000DE810D2605860ABDF8DE39BDF8DE9C54E7
:10F3B00026B89C5227B4098608BDF8DE8620BDF821
:10F3C000DE8608BDF8DE20A2DE548C80002508CC45
:10F3D00000087EEEF63232CE73D2BC73A225040D45
:10F3E00086FF39EC00847F9354250139E602DF560D
:10F3F0004FD3561820E4200108A6002AFB20DB3C4E
:10F40000DE52270738CC00087EEEF6DE548C8000F2
:10F4100024F2FE738CEC00847F26035D27B7189CD2
:10F42000543825D2FE738C200C09E6000886FF5064
:10F43000DF56D35618DC548A80A1002605E1012648
:10F4400001398C73D226E20D86FF3916A600081109
:10F450002601393637BDF5CC3332810D26EE39869B
:10F4600022BDEDD2260ABDF44B810D2601094F398C
:10F470008627BDEDD227EF817F260A8108260686E2
:10F480000D9DAB20E9393C964536848097449645DE
:10F49000847F97458614367A0045F6B59AC10A26C8
:10F4A0000E7D00522A09BDEF5D7C00447A0045F6CE
:10F4B000B59A4F18DF487F00477F0046BDF06DDEEC
:10F4C000522604DE542708D651377A004520E0D66C
:10F4D00051377B80442715964484012704862D9D4F
:10F4E000AB7A00452B1B86309DAB20F57A00452B6F
:10F4F0000686209DAB20F5964484012704862D9D29
:10F50000AB328114270C810A25028B078B309DAB0F
:10F5100020EF3297453839BDF5204FBDF44B0839FF
:10F52000EC00847FDD547F00527F0053080808867A
:10F53000049745BDF4868620BDF5CC39FE73A4BC86
:10F5400073A8260139A600083CFE73A6A70008FF91
:10F5500073A63820EAFE73AABC73AE26013909A649
:10F56000003CFE73AC09A700FF73AC3820EA3233CD
:10F57000DF5E38FF7394271838FF739A38FF739C47
:10F5800038FF739638FF739838FF739E38FF73A067
:10F590003736DE5E393233DF5E308CB6012405DE6D
:10F5A0005E7EF352FE7394271BFE73A03CFE739E97
:10F5B0003CFE73983CFE73963CFE739C3CFE739A33
:10F5C0003CFE73943C3736DE5E39860D369DAB3299
:10F5D00036810D2604860A9DAB32397D00932601C3
:10F5E000397D009E27FA7F0093BDF83F0E7D008C89
:10F5F000271A8EBFFDCC0000FD738EFD7394CC00E6
:10F6000064DD54CC0000DD523C7ECB04FE738C27BD
:10F6100027CEF63BBDF5CA4FBDF44BFE738CEC0014
:10F62000847FDD547F00527F00537F0045860AB7F8
:10F63000B59ABDF486BDF5CA7EC6FE425245414B21
:10F64000204154204C494E4520000F36BDF747322B
:10F65000843F8A8016BDF67CC6EFD71671DF17BDD2
:10F66000F74ED756BDF74ED757BDF73EC6FFD71654
:10F670000E39BDF67C71DF1771BF173971DF177155
:10F68000BF1771EF1772401772201771DF177210D2
:10F69000177220178608BDF771390F36BDF747324C
:10F6A000843F36C630BDF67232368AC016BDF67C4F
:10F6B000BDF6D70E01010F32843F8A4016BDF67C9D
:10F6C000D656BDF76FD657BDF76FBDF6D7C600BD8E
:10F6D000F672BDF73E0E3971EF1771DF1771BF1764
:10F6E000CE02627220170101010171DF170926F3B2
:10F6F00072401772201771DF1771BF1739B6C43007
:10F700008154270AC11C2706C1182702D643BDF71A
:10F7100047BDF718BDF73E390F9F688E00FF71BFD8
:10F72000177220175858588605BDF771C6EFD716BF
:10F7300071DF17BDF74E86FF97169E680E39961734
:10F74000840F8A80971739710F1772401739C602D4
:10F7500072201771DF177B101727015C7220175872
:10F7600024F171DF177B101727015C72201739868F
:10F77000085871DF17721017250371EF17722017E1
:10F780004A26EE39961ED6113784D0275684502744
:10F79000049612323BDE719612A7007B0176271287
:10F7A00081132605728076203A81112605717F76B5
:10F7B0002031810326037C0093098C728B2603CEB3
:10F7C000738BDF717D0075261A189373C140261361
:10F7D000FCB596B3B594C1FF27098613BDF8DE8644
:10F7E000FF9775328424812427013B7B01762723F0
:10F7F0007B8076271EDEAFBDF5DB71FB110E0101AC
:10F8000096431A914327F90F0927057B807626E74F
:10F81000717F76FEB596A600098CB4932603CEB50B
:10F8200093FFB5967D007726029713FEB596BCB57B
:10F8300094260471FB113B7204113B86FF97753CC3
:10F84000CE738BDF71DF7371FB11CEB593FFB5946F
:10F85000FFB596967527088611BDF8DE7F007538CE
:10F86000717F767F0093399674907239B6B597B0F0
:10F87000B59539DE643CDE663CDEB3EC00DD64EC5D
:10F8800002DD663CBDF02B38D664E700D665E701A3
:10F89000D666E702D667E70338DF6638DF643338B9
:10F8A000393C3736DCB33226CADE739C7126031A24
:10F8B00020F7A60036098C728B2603CE738BDF737C
:10F8C0009675270F189371C14026088611BDF8DE82
:10F8D0007F0075323338810326037A0093393C3731
:10F8E00036FCB596B3B594C1FF27F6FEB59432A7A2
:10F8F00000098CB4932603CEB593FFB5947204111E
:10F9000033383986209DAB86209DAB393B3B717FD8
:10F910001BDE6C08DF6CDC42C30001DD42DC40C949
:10F92000008900DD4096AE890097AE3B7B20112711
:10F93000FB971339860297908E00FDBDF94E1A1A77
:10F940001ACE0000DF42DF407F00AE7EC683861203
:10F95000971BB6C42E8B0C971C97637F00017F000A
:10F96000207F008B7F008A860A9711860597108674
:10F97000E09714868097178602979086FF971686E1
:10F980000397707F009186FF9780867EB7010FCC2A
:10F99000F90EFD011072401B0E86FF9777392A2061
:10F9A0002050433D2420413D2420423D2420463D1B
:10F9B0002420583D242040583D242053503D2420ED
:10F9C0004024DEAC3CCEF8DEDFAC0E860DBDF8DEAA
:10F9D000860ABDF8DECEF99EBDFA5A3C30EC091815
:10F9E00009BDFA6238BDFA5A3C30A606BDFA67383E
:10F9F000BDFA5A3C30A605BDFA6738BDFA5A3C300C
:10FA0000A604BDFA6738BDFA5A3C30EC0718BDFAB7
:10FA10006238BDFA5A3C30EC0718EC0018BDFA62A7
:10FA200038BDFA5A3C3018C3000A18BDFA6238BD16
:10FA3000FA5AFE7282BDFA62863DBDF8DEFE72821F
:10FA4000860836A60008BDFA678620BDF8DE324A71
:10FA500026F038DFAC3BBDF8DE08A600812426F690
:10FA600008393C328D013236444444448D0132849D
:0CFA70000F8B30813A25028B077EF8DEF8
:10FFCA007EF7187EF7477EF73E7EEF827EEF967EBB
:10FFDA00F8677EF8A17EF8DE7EF83F7EF6FD00C364
:10FFEA000100010FF90CF784010301060109010C54
:06FFFA00F9C2F90DF93413
:00000001FF
